:100000000C94DE010C9416020C9416020C94160249
:100010000C9416020C9416020C9416020C94160200
:100020000C9416020C9416020C94F8210C94CC2219
:100030000C94181C0C9416020C9416020C941602C4
:100040000C9416020C9416020C9416020C941602D0
:100050000C9416020C949F1C0C9416020C9416021D
:100060000C9416020C9416020C9416020C941602B0
:100070000C9416020C9416020C9416020C941602A0
:100080000C9416020C9416020C9416020C94160290
:100090000C9416020C9416020C9416020C94160280
:1000A0000C9416020C9416020C9416025300540081
:1000B000550056005F006000610057005C005D0065
:1000C0005E00570059005A005B0058006200620051
:1000D000630058000100010001000100010001005F
:1000E0000100010001000100010001000100010008
:1000F00001000100010001000100010001000100F8
:1001000001000100010001000100010001000100E7
:1001100001000100010001000100010001000100D7
:1001200001000100010001000100010001000100C7
:1001300001000100010001000100010001000100B7
:1001400001000100010001000100010000000000A9
:10015000000000002A2B2800000000000000000022
:100160000000000000000029000000002C1E3420C8
:10017000212224342627252E362D3738271E1F20EE
:100180002122232425263333362E37381F04050633
:100190000708090A0B0C0D0E0F1011121314151677
:1001A0001718191A1B1C1D2F3130232D3504050675
:1001B0000708090A0B0C0D0E0F1011121314151657
:1001C0001718191A1B1C1D2F3130354C0000000068
:1001D000000000000000000000000000000000001F
:1001E000000000000000000000000000000000000F
:1001F0007E0F00D4FFFFFFC7000000780C03530000
:100200006F00790075007A00000026036100690024
:10021000300033002000440065007300690067006F
:100220006E002000530074007500640069006F00C8
:1002300000000403090409025B00030100A0FA099D
:100240000400000103010100092111010001224005
:1002500000070581030800010904010002030000F2
:10026000000921110100012222000705820320005C
:100270000107050303200001090402000103000037
:100280000009211101000122B600070584032000A6
:1002900001120100020000000803A1180001000182
:1002A0000200010660FF0961A1010962150026FF35
:1002B000009520750881020963150026FF0095202E
:1002C00075089102C005010902A10185020901A179
:1002D00000050919012908150025019508750181F6
:1002E000020501093009311581257F9502750881C4
:1002F0000609381581257F950175088106050C0AC8
:1003000038021581257F950175088106C0C0050159
:100310000980A101850319012AB700150126B7003C
:10032000950175108100C0050C0901A10185041912
:10033000012AA002150126A002950175108100C0B6
:1003400005010906A1018506050719E029E7150041
:1003500025019508750181020507190029EF15008F
:10036000250195F0750181020508190129059505FA
:1003700075019102950175039101C005010906A15E
:1003800001050719E029E715002501950875018188
:10039000029501750881010507190029FF1500263E
:1003A000FF009506750881000508190129059505C6
:1003B00075019102950175039101C00011241FBEC2
:1003C000CFEFDAE0DEBFCDBF04B603FE18C08091E8
:1003D000930290919402A0919502B0919602873079
:1003E000904BA740B04B59F4109293021092940294
:1003F0001092950210929602E0E0F8E3099511E060
:10040000A0E0B1E0E2E4FBE402C005900D92A23965
:10041000B107D9F722E0A2E9B1E001C01D92A339EA
:10042000B207E1F70E94F4100C9437250C940000F9
:1004300084E0089581E0089581E008950E941C02FF
:10044000089508950E9421020895A5E0B0E0EBE22E
:10045000F2E00C94A32449835A8330919901898155
:100460009A81311119C0662399F0222389F00E94E4
:100470001808182F682F89819A810E94F5076981D1
:100480007A81812F0E9404192596E3E00C94BF2401
:100490000E940608182FF3CF0E94180869817A81FC
:1004A000F1CFFC01262F40815181628173818481CB
:1004B0000E942502089581E00895CF93DF93EC0117
:1004C00060E00E945102BE010E942202DF91CF91A2
:1004D0000895E1E0F0E0DF0102C0AA0FBB1F6A95BA
:1004E000E2F7BD01DF0102C0AA0FBB1F4A95E2F788
:1004F0006A2B01C0EE0F2A95EAF7962F98239613E0
:1005000002C08E2B0895E0958E230895242F462F48
:10051000682F8091A3010E9469020E9455070895E7
:100520000E94AE0F08950E94B20F089508950E9490
:10053000E7060E9496022FEF84E39CE02150804062
:100540009040E1F700C0000008950E9497020E94C9
:10055000C31C08950E9497020E94E71C08950F9300
:100560001F93CF93DF938C0161E00E945102EC0155
:10057000B8010E94EA13811106C080E0DF91CF919B
:100580001F910F910895B801CE010E941E02882389
:10059000A1F3B801CE010E944A1A882371F3B80171
:1005A000CE010E94D914882341F3B801CE010E94E4
:1005B000BC19882311F3F8018281882361F0CA35C0
:1005C000FDE5DF0701F158F4C115ECE5DE0791F018
:1005D000CE3DDC4591F0C8010E941A02CFCFCC3548
:1005E0008DE5D80769F090F0C73ADD45A1F70E9484
:1005F000AA02C3CF0E94A502C0CF0E94D10CF7CFA0
:100600000E940B0CE8CF0E94150CE5CF0E94190C3C
:10061000E2CF0E94F51B0E94260308950E942A0340
:100620000E94FA1B089508950E941303089581E023
:1006300008950E94170308950895CF93C82F0E942C
:1006400014038C2F0E941903CF91089580E00E941B
:100650001D0308950E94A61A0E941D030895CF93BA
:100660000E94A61AC82F809194018C1779F0C0932C
:1006700094010E94841C609395017093960180936D
:100680009701909398018C2F0E941D03CF9108959C
:10069000ABE0B0E0EEE4F3E00C94A4244F83588781
:1006A00069877A878B8761110E94560B1E821D8293
:1006B00085E0FE013796DE01119601900D928A9534
:1006C000E1F78C819D81892B61F449815A816B818D
:1006D0007C818D819E810E947F0A2B96E2E00C94A2
:1006E000C02489819A8189238F3F79F3CE010196B5
:1006F0000E945B028111E9CFF0CFFC0180819181E2
:100700000E9445080895CF93C82F8823C9F08238E6
:10071000C9F40E94A61A81FD13C089E30E940E0B42
:100720000E94770B2FEF87EE93E02150804090409E
:10073000E1F700C0000089E30E94160B0E94770BCE
:10074000CF9108958338A1F40E94A61A80FDF8CFB6
:1007500083E50E940E0B0E94770B2FEF81EE94E051
:10076000215080409040E1F700C0000083E5E4CFD5
:100770008438A1F40E94A61A82FDE2CF87E40E9489
:100780000E0B0E94770B2FEF81EE94E021508040FA
:100790009040E1F700C0000087E4CECF8CEF8C0FD3
:1007A000813AB8F48C2F0E9478178111C9CF6C2F31
:1007B00080910001909101010E941B1B882329F068
:1007C0008C2F0E94160B0E94770B8C2F0E940E0B11
:1007D000B5CF80E28C0F883048F4C77081E001C04B
:1007E000880FCA95EAF70E94390BA8CFEBE5EC0F0A
:1007F000E33040F4F0E0EB5BFE4F808190E00E943C
:10080000DB1A9ECFE8E5EC0FE73150F4F0E0EE0F95
:10081000FF1FE95EFE4F808191810E94F11A90CF07
:10082000C03F08F48DCF8C2F0E9478110E944B128C
:1008300087CF882309F455C0823879F40E94A61A1C
:1008400081FF4FC089E30E940E0B0E94770B89E362
:100850000E94160B0E94770B0895833859F40E946A
:10086000A61A80FF3EC083E50E940E0B0E94770B04
:1008700083E5EECF843859F40E94A61A82FF31C076
:1008800087E40E940E0B0E94770B87E4E1CF9CEF78
:10089000980F913AE8F290E2980F983050F48770F0
:1008A00091E001C0990F8A95EAF7892F0E943F0BCA
:1008B000D1CF9BE5980F933028F490E080E00E9420
:1008C000DB1A089598E5980F973128F490E080E0BE
:1008D0000E94F11A0895803F20F00E94D2110E94D8
:1008E0004B1208951F93CF93DF93182FEB010E94B3
:1008F0008303209739F4812F0E941904DF91CF914F
:100900001F9108958FE99FE00197F1F700C0000063
:100910002197EFCF70E060E0893311F460E570E07B
:100920000E9472040895882321F00E94390B0E94CE
:10093000770B0895882321F00E943F0B0E94770BCC
:100940000895B0E0A0E0E7EAF4E00C949D246C0187
:10095000D62FC72FFC011281F580F2949FE0F92277
:100960000E942F0BE82E8823B9F0E12E1123A1F06D
:100970008C2F807F803421F080E28D0F8830D0F082
:100980008091770282FF16C082E00E94DA0B0E94FB
:100990002F0B91E0E82EE926BC2EB2948FE0B8220E
:1009A000FBE0FB1508F468C0EB2DF0E0E75CFA4DC6
:1009B0000C948724E12CF0CF0C2F0F70C07F11F026
:1009C0000295007F112399F0002359F080E28D0FEA
:1009D000883010F0D11107C0802F0E94390B0E947F
:1009E000770B8D2F41C0802F0E94490BF8CF8D2FA0
:1009F0000E941904002309F43FC080E28D0F883063
:100A000010F0D11104C0802F0E943F0B03C0802F33
:100A10000E944F0B0E94770B2FC00C2F0F70C07FCE
:100A2000C03211F00295007FDD2381F0D13009F44E
:100A300063C0112309F46DC0FF2009F463C0F601FF
:100A4000858180FFCECF8F7085835CC080917702D7
:100A500082FD33C0112359F0002329F0802F0E941A
:100A6000390B0E94770B80E00E94830305C080E071
:100A70000E9419040111C7CFEB2DE850FF0B3497EA
:100A800020F40E94A61A0E941D03EE2089F00E9405
:100A90002B0B80FD0DC0F60112820E94250B0E94D7
:100AA0006907C6010E94A7060E94250B0E947507D0
:100AB000CDB7DEB7E9E00C94B924112389F0F11029
:100AC00006C00E94590B802B0E949304D5CF21E0D1
:100AD000F212F7CF0E94590B802B0E94600BCCCFF3
:100AE000F11006C00E946D0B802F0E949A04C4CFA3
:100AF00031E0F31609F2F6CF112331F085E08F15BE
:100B000008F4BACF802FE0CF94E09F1508F4B4CF5B
:100B1000EBCFFF2049F3D93349F4FFEF27EE33E061
:100B2000F15020403040E1F700C000008D2F0E94BE
:100B30001904A2CF8C2F86958695837069F0813039
:100B400009F09ACF8D2F9C2F9370111102C090E065
:100B500080E00E94F11A90CF8D2F9C2F937011117D
:100B600002C090E080E00E94DB1A86CF8D2F112317
:100B700029F00E9478110E944B127ECF0E94D21160
:100B8000FACF8C2F837079F5111176CF4D2F4295C6
:100B900046954770440F440F8D2F8F70042E01C06F
:100BA000880F0A94EAF72D2F2071D4FF07C02FE099
:100BB00030E001C0220F4A95EAF72095C695C69508
:100BC000C370822BC23049F058F4C13019F00E9432
:100BD000430752CF0E943D074FCF0E9449074CCF99
:100BE0000E943A0749CF8695112311F08C2F81700E
:100BF000882309F441CF4D2F429546954770440F05
:100C0000440F8D2F8F70042E01C0880F0A94EAF7CD
:100C10002D2F2071D4FF07C02FE030E001C0220F3C
:100C20004A95EAF72095C695C695C370822BC230C7
:100C300049F058F4C13019F00E9494071DCF0E946A
:100C40008E071ACF0E949A0717CF0E94550714CF1C
:100C5000CF70112329F08C2F0E9469078D2F34CF7C
:100C60008D2F0E949A048C2F0E94750705CFD23FCA
:100C700051F160F4D03FB9F0D13F81F0112309F474
:100C800049C0F110AECE8C2F8F7121C0D33F11F12E
:100C9000D43FA1F78091770282FD26C08C2F8F71FF
:100CA000112311F314C0112349F084E08F1508F4C7
:100CB000E3CE8C2F8F710E948207DECE95E09F15C8
:100CC00008F4DACEF6CF8C2F8F711111CDCF0E94A0
:100CD0006907D2CE112329F08C2F8F710E946007F3
:100CE000CBCE0E945C07C8CE112349F0CF718C2F68
:100CF0000E94690763E08C2F0E94BC0BBDCE81E08F
:100D00000E94DA0BE1E0EF1508F0B6CE82E00E9417
:100D1000DA0BB2CEF110FFCE8C2F8F71A5CF0F93CF
:100D20001F93CF93DF93EC01688179818A810E94C0
:100D300050088C010E94A0070E943907B801CE011B
:100D40000E94A104DF91CF911F910F910895CF933D
:100D5000DF93EC018B819C81892B29F0888199811B
:100D600089238F3F51F4DF91CF910895CE010E94E6
:100D70008F06CE010E945D02F6CFCE010E94AF0227
:100D80008111F4CF0E942F0B882369F38A81882375
:100D900051F38091770282FFE6CF82E00E94DA0B66
:100DA000E2CF90E080E00E94DB1A90E080E00E94B9
:100DB000F11A0E94560B0E94770B0E9467120E9444
:100DC0004B1208950E941E0B0E94D10608950E94A6
:100DD000460B0E94E206089592959F70963091F01E
:100DE00058F4925F9F70923058F4803F19F030F4BD
:100DF000883E30F481E008959A5FF4CF843FD1F3C8
:100E000080E00895883EB0F3813FD1F7F3CFFC0135
:100E100083819481892B29F08081918189238F3F5F
:100E200011F480E00895808191810E9445080E941C
:100E3000EC060895A5E0B0E0E0E2F7E00C94A4240D
:100E40002596E2E00C94C024A6E0B0E0EAE2F7E0E8
:100E50000C94A4242696E2E00C94C02408950E94E9
:100E60002E0708950E942F078093A4010E94D106A7
:100E7000089508950E94320708959091A401892B46
:100E80000E94320708959091A40189230E9432079D
:100E900008959091A40189270E94320708950E9425
:100EA0002E0708950E944F0708950E9452078093CD
:100EB000A3010E94D106089580E00E94550708957D
:100EC00091E001C0990F8A95EAF7892F0E94550792
:100ED000089521E030E001C0220F8A95EAF7809161
:100EE000A301822B0E945507089521E030E001C044
:100EF000220F8A95EAF720958091A30182230E9410
:100F00005507089521E030E001C0220F8A95EAF7E5
:100F10008091A30182270E94550708959091A30113
:100F2000892B0E94550708959091A30189230E945F
:100F3000550708959091A30189270E9455070895A8
:100F40000895262F277091E001C0990F2A95EAF79E
:100F500023E0769567952A95E1F7FB01EE0FFF1FD9
:100F6000E60FF71FE40FF51F50E040E0682F70E038
:100F70008191DF0111979B01042E02C036952795C0
:100F80000A94E2F7217021952827292328272C93FA
:100F90004F5F5F4F4330510559F70895A82FA77051
:100FA00023E0969587952A95E1F7FC01EE0FFF1F48
:100FB000E80FF91FE60FF71F50E040E080E02191B5
:100FC00030E00A2E02C0369527950A94E2F7217088
:100FD0003327042E01C0220F0A94EAF7822B4F5FB9
:100FE0005F4F4330510559F70895262F953068F427
:100FF000843058F434E0939FB0011124680F711DC0
:101000004AE951E0822F0E94A1070895953070F4BB
:10101000843060F444E0949F900111246AE971E007
:10102000820F932F911D0E94CE07089580E00895AE
:10103000CF92DF92FF920F931F93CF93DF936C01B8
:101040000091A3018091A401082BC7E0D0E010E03B
:10105000FC2EC8010C2E02C0959587950A94E2F7E4
:1010600080FD0CC02197A0F7F12C8F2DDF91CF913F
:101070001F910F91FF90DF90CF900895B6018C2FB4
:101080000E948C0E019771F3F0CFCF93DF93EC01A8
:101090000E941808BE010E948C0EDF91CF91089526
:1010A0001F93CF93DF93EB0190919901992339F02E
:1010B000CB010E944508DF91CF911F9108958823AD
:1010C00069F0CB010E941808182F682FCE010E94EA
:1010D000F507BE01812F0E948C0EEDCFCB010E943F
:1010E0000608182FF6CF1F93CF93DF93C091A50169
:1010F00016E08091A6018C1304C0DF91CF911F915F
:101100000895D0E01C9FF0011D9FF00D1124E955BA
:10111000FE4F4081518162817381848195810E945B
:1011200024072196C770E5CF4091D7015091D8018F
:101130006091D9017091DA018091DB019091DC011D
:101140000E94240708951F93CF93DF938091DC01C1
:10115000807F09F049C08091D901882309F444C0F7
:101160008091A501C091A6016091D7017091D8012D
:10117000A091DA01B091DB01D62FD72316E0C81772
:1011800099F190E0109711F0DF3F19F40196877004
:10119000F6CF189F9001199F300D1124F901E955E0
:1011A000FE4F41814713F2CF40814613EFCF42817A
:1011B0004111ECCF438154814A1B5B0B483C5105E4
:1011C00028F78091DC018F7080618093DC01F90148
:1011D000E455FE4F80818F708061808387ED91E0C0
:1011E0000E94A7060E947308DF91CF911F91089576
:1011F000A1E1B0E0EEEFF8E00C949C248C0185E0D6
:10120000F801DE011D9601900D928A95E1F7F80133
:10121000E28087EDC82E81E0D82E6091DA017091CE
:10122000DB016115710509F44EC19091D701209140
:10123000D801892F82238F3F09F445C14081518114
:10124000A380B480F090D901F501E61BF70BFF20D5
:1012500009F4EAC08091DC01382F307FE83CF105C9
:1012600008F0A3C031116DC0FE2C251316C09413D5
:1012700014C0E11012C08F7080618093DC010E9465
:101280009408C6010E94A7068091DC01F8018583BD
:101290008F2D6196EAE00C94B824A114B10429F0D2
:1012A000842F85238F3F09F027C180E0F82FF1704C
:1012B000DF2E80FF3CC08091A5012091A60136E081
:1012C000821315C04D875E878D859E850E944508D7
:1012D000292F22952F702230F0F0243018F59F70BE
:1012E000F1F0F8019581907FD1F4D12C1EC090E0EF
:1012F000389FF001399FF00D1124E955FE4F6181AF
:10130000651306C06081641303C06281E6120FC0DA
:1013100001968770D5CF9F7011F0882331F3805EDE
:10132000883018F3C8010E94A706FD2CB1CFEE202B
:1013300009F4AECF8091DC0181608093DC01F12C57
:10134000A7CF251306C0941304C0F801EE2009F4BA
:1013500087C0C8010E940707882319F1EE2009F110
:101360008091DC01803270F02091D7013091D8015A
:1013700038872F831986BB86AA868C87CE0107966D
:101380000E94A70686E0F801A7EDB1E001900D925A
:101390008A95E1F70E94A3080E949408FF24F39421
:1013A00077CFC8010E94A706F9CF311113C07A2D5B
:1013B000B98AA88A6E2D89890E941A0787ED91E063
:1013C0000E94A70686E0F60111928A95E9F70E942D
:1013D0009408B5CF25130FC094130DC0E1100BC0B6
:1013E000F8018583C8010E94A70686E0F6011192E4
:1013F0008A95E9F74DCFC8010E940707882389F233
:10140000EE2079F28091DC01803208F4BBCF20918C
:10141000D7013091D8013A8329831B82BD82AC82E7
:101420008E83CE010196ACCFE83CF10508F03EC0BA
:10143000FE2CEE2009F4B5CF25132AC0941328C042
:101440008091DC0180FD1BC0982F907FC1F0F801D6
:101450008583903F31F0982F907F905F8F70892B1C
:101460008583C8010E94A70686E0F801A7EDB1E0D8
:1014700001900D928A95E1F70E94940809CF86E0C9
:10148000F801A7EDB1E001900D928A95E1F700CF48
:10149000C8010E940707811175CF8091DC0181602E
:1014A0008093DC01C8010E94A706F2CE7A2DB98A8A
:1014B000A88A6E2D89890E941A0786E0F60111928A
:1014C0008A95E9F7D9CFEE2009F46BCFC8010E94C5
:1014D0000707F82E882309F464CF86E0F801A7ED0A
:1014E000B1E001900D928A95E1F787ED91E00E94BD
:1014F0007D030E94A308C0CF81E08E25D7CEACE04B
:10150000B0E0E5E8FAE00C94A3244F83588769879C
:101510007A878B879C87CE0107960E94F8088823DC
:1015200069F08A859B85892B39F04F815885842FF6
:1015300085238F3F09F06BC016E05FC086E0FE0197
:101540003796DE01119601900D928A95E1F78A8512
:101550009B85892B89F38F81988589238F3F61F340
:101560002091A60130E0C90101968770992740912A
:10157000A5014817190671F40E94E7061092A6010A
:101580001092A50186E0E7EDF1E0DF011D928A955A
:10159000E9F7D2CF96E0929FD001939FB00D11242E
:1015A000A955BE4FFE01319601900D929A95E1F733
:1015B0008093A6010E947308BFCF819FC0011124B0
:1015C00089559E4F0E94F8088823E9F0E091A50113
:1015D0001E9FF0011124E955FE4F40815181628127
:1015E0007381848195810E9424078091A50190E0F8
:1015F0000196877099278093A5018091A50190910C
:10160000A6018913DACF2C96E3E00C94BF246985F8
:101610007A858B859C850E9424078ECF682F8091C8
:101620000001909101010E949B1B0895682F8091F9
:101630000001909101010E94A91B08958091000171
:10164000909101010E94B71B08958091FD0185953D
:101650008595859508958091FD01877008959091F5
:10166000FD01977081E009F480E0089580912002E7
:10167000089590912002892B8093200208958095EF
:1016800090912002982390932002089510922002B6
:10169000089590911F02892B80931F0208958095D1
:1016A00090911F02982390931F02089510921F0299
:1016B00008958091FE01089508950E945C0B08959D
:1016C0009091770292FF08C09091FE01981721F047
:1016D0008093FE010E945D0B08958091FE01882396
:1016E00029F01092FE0180E00E945D0B0895CF93D7
:1016F000DF93E0910001F09101018091200280834D
:10170000E0910001F0910101808190911F02892BED
:1017100080839091FE01992381F0E0910001F09186
:1017200001018081892B80838091000190910101CA
:101730000E94071B81110E946D0BC0910001D09186
:10174000010140E250E06DED71E0CE010E94DF2426
:10175000892B59F080E2FE01ADEDB1E001900D92D0
:101760008A95E1F7CE010E94B31ADF91CF910895D7
:1017700008950E94B80B08959091770292FF11C0CE
:1017800098E0899F90011124622B6093FD010E94D3
:1017900069078091FD018595859585950E94B90B16
:1017A00008950E94690708951092FD0180E00E944B
:1017B000B90B08959091FD01809589238093FD01D7
:1017C000282F277091F4282F082E000C330B921726
:1017D000130659F09091770292FF07C08595859581
:1017E00085950E9475070E94D40B08959091770209
:1017F00092FB222720F9281769F080FB92F9909339
:10180000770280917602909177020E94480C82E0E4
:101810000E94DA0B08958091770282FB882780F975
:1018200091E089270E94F60B089581E00E94F60B53
:10183000089580E00E94F60B08956FEF7FEF90E02F
:1018400080E00E942125089590E080E00E94FD2420
:10185000883E9E4F19F40E948513089580E00895F4
:1018600082E090E00E94F524089583E090E00E94D9
:10187000F5240895CF9384E090E00E94F524C82FCA
:1018800082E290E00E94F524982F8C2FCF9108954A
:10189000CF93C92F682F84E090E00E9403256C2F1E
:1018A00082E290E00E940325CF910895AB01BC0134
:1018B0008FE090E00E9415250895AB01BC0183E103
:1018C00090E00E941525089560E070E0CB010E9431
:1018D0005D0C089560E070E0CB010E94560C0E9400
:1018E000640C089568EE7EEF90E080E00E94212570
:1018F00060E082E090E00E94032560E083E090E0F9
:101900000E9403251092A40160E084E090E00E9410
:10191000032564E082E290E00E94032560E085E018
:1019200090E00E94032560E086E090E00E9403259D
:101930006FEF87E090E00E94032540E050E0BA019D
:1019400088E090E00E94152560E08DE090E00E9424
:10195000032540E050E0BA0188E190E00E9415259F
:1019600060E087E190E00E94032540E050E0BA018A
:101970008CE190E00E94152570E060E080E290E04C
:101980000E94212540E050E0BA0188E190E00E94E9
:10199000152580E00E949E130E94CD130E946A0CC0
:1019A00008950E94720C0895682F8EE090E00E94C6
:1019B000032508950E94841C60932C0270932D02CD
:1019C00080932E0290932F02609328027093290235
:1019D00080932A0290932B020895089508950E94FF
:1019E000EE0C089508950E94F20C089586E79FE09A
:1019F0000E949C1A0E94ED0C0E94EF0C089581E059
:101A000008950E94FF0C0895089508950E94040D02
:101A10000E94050D08950E94920F0E941C030895D4
:101A20000E946F1C0E94DD130E9457100E940B0D34
:101A30000E94F30C0895AAE0B0E0E1E2FDE00C940E
:101A40009C240E946D1083E2A82E82E0B82E7501BE
:101A500010E0F70101917F01812F0E94B50F1F5FF8
:101A6000153009F440C00817A1F38091300281FDC0
:101A70000E94BB0F0E94010DC82E10E0812F0E9412
:101A8000B50F082FF50181915F01081731F1D02EB4
:101A9000D826F12CEE24E3948D2D8E21B1F0CC20AC
:101AA000A1F0FE821F8391E0802F8E2109F490E047
:101AB00098870E94781C8160782F9A8789874E8149
:101AC0005F8168858A850E944803F394EE0CF4E0F8
:101AD000FF12E2CFF501319700831F5F153071F6D9
:101AE0000E94DA0C20C00813C0CF0E94781C8C0121
:101AF000809121029091220208171907A1F08FEF1F
:101B000089838A831B820E94781C8160782F9D8341
:101B10008C8349815A816B818D810E944803109387
:101B20002202009321020E9489120E942F032A960A
:101B3000EAE00C94B824CF93DF930E94910EEC015D
:101B4000811521E5920708F042C0811530E5930721
:101B500008F09FC0883E910530F5803E910508F061
:101B600094C0883A910588F4853A910508F086C0BA
:101B70008130910509F489C0009709F486C0049763
:101B800008F083C0D0E0C0E080C08F3B9105D0F763
:101B9000C85AD0E0CC0FDD1FC85BDE4F0990D8815A
:101BA000C02DD46472C0811540E2940750F4C11571
:101BB00081E0D80708F069C0C03FD10518F3D065AF
:101BC00064C081159044F0F2DF70D06A5EC0811568
:101BD00035E5930718F5811544E5940708F085C0AD
:101BE000C11583E5D80708F06CC0C11522E5D207FE
:101BF00008F462C0CE018370992721E030E002C072
:101C0000220F331F8A95E2F7C695C69580E2C89FDA
:101C1000E0011124C22BD32BDC6837C0811539E5D4
:101C20009307A8F4811548E5940708F063C0C1152F
:101C300086E5D80708F0A6CF8C2F0E94330FC82F57
:101C4000D0E0DC2FCC27CC27DF71D0621EC08115FD
:101C50002AE5920708F453C090568115904208F087
:101C600091CF8D2F8F710E94330F90E0982F88278E
:101C700088279F719C012C2BE901E7CFC55AD0E042
:101C8000CA58DE4FC881D0E0D064CE01DF91CF9139
:101C900008958370992721E030E002C0220F331F9E
:101CA0008A95E2F7C695C69540E2C49FE0011124EB
:101CB000C22BD32BDD68E9CFDC2FCC27C16FD06AD4
:101CC000E4CFCE018370992721E030E002C0220FDB
:101CD000331F8A95E2F7C695C69540E2C49FE0019E
:101CE0001124C22BD32BDA68D0CFD82FCC27C46FC6
:101CF000D06ACBCFD82FCC27C06FD06AC6CF8F7019
:101D00000E94330F34E0D695C7953A95E1F7CF702E
:101D10009C2FEC01D069B9CF0E9404190E949B0D41
:101D2000089582389105B9F1B0F48133910509F431
:101D30007DC048F48932910509F46DC08A3291055D
:101D400009F47BC008958533910509F45FC0893398
:101D5000910509F10895833E9105D9F138F4803E4B
:101D6000910529F1823E910579F10895863E91050C
:101D7000D9F1873E910509F43EC0843E910541F5B5
:101D80002091770221FF24C08091760284FD19C042
:101D900087EE90E0089520917602237009F05AC0F2
:101DA0002091770223FF14C089E290E008952091EA
:101DB000760220FD38C03091770230FF09C024FF41
:101DC00043C090E080E008952091760222FDF7CF95
:101DD00008952091760222FD3AC03091770230FDBD
:101DE00039C024FFF5CFEDCF2091760223FFF0CF4D
:101DF00024FDE7CFCDCF2091760223FD2EC0309178
:101E0000770231FFEECF84EE90E0089520917602C4
:101E100025FFDECFC9CF2091760225FD21C020917C
:101E2000770223FFD5CF89E390E0D2CF20917602CD
:101E300026FFCECF8AE290E008952091760226FF19
:101E4000C7CF81E390E0089583EE90E0089582EE9D
:101E500090E0089580EE90E0089586EE90E0089579
:101E600085E390E008959091760292FF06C0282FB6
:101E700028712830F9F4877F846093FF06C0282FEB
:101E800028712831F1F4877E84612091770220FF48
:101E900006C0382F38713830D9F4877F816021FF30
:101EA00006C0282F28712831D1F4877E816194FDE6
:101EB000877E0895282F24712430F9F68B7F88605F
:101EC000DCCF282F2471243101F78B7E8861DDCF90
:101ED000382F3171313019F78E7F8860E0CF282F8D
:101EE0002171213121F78E7E8861E1CF80E0089554
:101EF0000E941D0C08950E946D108FE39CE90197CC
:101F0000F1F700C000000E946D1080E00E94B50F44
:101F100080FF04C00E94780F0E94C31C08950E9495
:101F20007B0F08950E94240C811102C00E94D10CE5
:101F30000E94300C809330020E943A0C90937702FA
:101F4000809376020E948F0F0E94350C0E943A0700
:101F50008091A3010E945207089508950E94AD0F39
:101F6000089508950E94B10F0895E82FF0E0E35816
:101F7000FD4F80810895089580EA8A95F1F70895CC
:101F800000C008950E94BC0F0895F894E82FE295D0
:101F9000EF70F0E031A1282F2F7081E090E001C0B8
:101FA000880F2A95EAF7982F9095932391A392A1F1
:101FB000892B82A378940895CF93DF93CDE7D1E066
:101FC00089918F3F11F00E94C50F81E0C238D80778
:101FD000B9F784EF0E94C50F83E30E94C50F87E91C
:101FE0000E94C50F85E30E94C50FDF91CF91089530
:101FF000B0E0A0E0EEEFFFE00C949E24EC01D62EC2
:10200000062F10E0C80183589E4F7C01FC0180819F
:102010008F3F09F445C0F894E82FE295EF70F0E0A7
:1020200091A18F7021E030E001C0220F8A95EAF77C
:10203000892F822B81A382A12095282322A3789423
:102040000E94C00FE9E7F1E04DE751E031E0C12C1B
:1020500021912F3F51F1A22FA295AF70B0E0909641
:102060008C9190E02F7002C0959587952A95E2F7A4
:1020700080FD1BC0832FC82A330F4E175F0741F71F
:10208000F70180818F3F11F00E94C50F61E0C11000
:1020900001C060E08D2D0E94C20FC00FD11FC88209
:1020A000CDB7DEB7E8E00C94BA2480E0E4CF0E941C
:1020B000DC0F85E0EDE7F2E0DF01982F1D929A95A5
:1020C000E9F7E8E7F2E0DF011D928A95E9F785E09C
:1020D0000E94A8100E9490020895A5E0B0E0E3E7F6
:1020E000F0E10C94A1248E010F5F1F4F85E0F801F1
:1020F00011928A95E9F7F12C6F2DC8010E94F80F13
:10210000F394F5E0FF12F8CF45E050E0B80188E71E
:1021100092E00E94DF2421E0009709F420E0892B5F
:1021200041F085E0F801A8E7B2E001900D928A95B0
:10213000E1F745E06DE772E088E792E00E94A910C0
:10214000182F0E949302812F2596E5E00C94BD2460
:102150000895CF92DF92EF92FF920F931F93CF9348
:102160006C017B01042F222349F081E0809333022C
:102170000E94781C9093320280933102C091330206
:10218000C1110AC0C0E08C2FCF911F910F91FF9019
:10219000EF90DF90CF9008958091310290913202BC
:1021A0000E94901C059770F310E0A801B601C701CA
:1021B0000E94DF24892B41F0A801B601C7010E94CB
:1021C000EC2410923302DFCFC0E0FBCF0E94D21E7E
:1021D0000E94100D0E94DF1E08950E94E41E0E94BE
:1021E0001B0D0E94FE1E08950E94111C0E94B81E25
:1021F0000E94F60C0E94E6100E94ED100E94060D4F
:10220000FBCF80913A0280FF0DC06091070170E022
:10221000660F771F6038710570F56115710569F1FA
:10222000862F089581FF07C06091070184E0689FB1
:10223000B0011124EFCF6091070182FD0AC08091A7
:1022400039028823A9F020910601609107018217C5
:1022500010F088E0ECCF869FC001112433E0880F96
:10226000991F3A95E1F7622F70E00E947324D2CF54
:1022700068E070E0D5CF8FE7089581E00895809100
:102280003A0280FF0CC06091030170E0759567957C
:10229000759567956115710549F1862F089581FF40
:1022A00006C06091030170E075956795F3CF60916A
:1022B000030182FD0BC0909138029923A1F0609137
:1022C000020180910301961738F0682F70E06038A2
:1022D000710500F38FE70895899FC001112470E014
:1022E0000E947324F4CF61E070E0D7CF81E00895BD
:1022F000803F31F40E940111819580933E02089540
:10230000813F19F40E940111F8CF823F31F40E94FD
:102310000111819580933D020895833F19F40E9435
:102320000111F8CF893F29F40E943F1180933F02A9
:1023300008958A3F21F40E943F118195F7CF8B3F8A
:1023400031F40E943F1181958093400208958C3FA3
:1023500019F40E943F11F8CF9CE0980F953070F46B
:10236000845F990B21E030E001C0220F8A95EAF7E3
:1023700080913C02822B80933C0208958D3F31F482
:1023800080913A02816080933A0208958E3F21F451
:1023900080913A028260F7CF8F3FB9F780913A027D
:1023A0008460F1CF40913D02803F59F480913E021C
:1023B00087FF0DC010923E0241110BC010923902EE
:1023C00008C0813F81F480913E0218169CF344239B
:1023D00081F080913F0290914002892B09F05AC010
:1023E000109238020895823F49F447FFF0CF1092CF
:1023F0003D0280913E028111ECCFE0CF833F19F482
:102400001416ACF3E4CF90913F02893F29F41916DA
:10241000F4F610923F02DBCF8A3F19F497FFD7CF33
:10242000F8CF909140028B3F29F497FFD0CF1092C4
:102430004002CDCF8C3F19F41916CCF3C8CF9CE0E5
:10244000980F953090F4845F990B21E030E0B9014A
:1024500002C0660F771F8A95E2F7CB0180959091B5
:102460003C02892380933C02B2CF8D3F31F48091AE
:102470003A028E7F80933A02AACF8E3F21F4809158
:102480003A028D7FF7CF8F3F09F0A1CF80913A02BA
:102490008B7FF0CF08950E94781C9C0190913D02A3
:1024A00080913E02982B21F0309337022093360220
:1024B00090913F0280914002982B21F03093350299
:1024C000209334028BE392E00E94CD1A089586E0B7
:1024D000EBE3F2E0DF011D928A95E9F710923902F1
:1024E0001092380210923A020895FC018281811103
:1024F0000EC0838181110BC08481811108C091E0DD
:102500008581811101C090E0892F8170089581E05B
:10251000FCCFA6E0B0E0EFE8F2E10C94A32486E063
:10252000EBE3F2E0DE01119601900D928A95E1F75E
:1025300010923D0210923E0210923F021092400211
:102540008B819C81892B89F0809136029091370292
:102550000E94901CAC01909139029923C9F180919D
:1025600008018417150608F440C08D819E81892BCF
:1025700091F080913402909135020E94901CAC0140
:1025800090913802992309F471C080910401841755
:10259000150608F479C0BE016F5F7F4F8BE392E0B0
:1025A0000E94C91B811105C08BE392E00E94751245
:1025B00081110E944B1286E0FE013196ABE3B2E03E
:1025C00001900D928A95E1F72696E3E00C94BF24E2
:1025D000209109018AE0289F9001112424173507D2
:1025E00020F69F5F9093390202C09F3FD1F71B8175
:1025F000112359F00E9401119FEF11160CF491E084
:10260000899F802D112480933D021C81112359F054
:102610000E9401119FEF11160CF491E0899F802D0B
:10262000112480933E0230913D02332309F49DCF63
:1026300020913E02222309F498CF45EB3403C001D8
:102640001124992359F090933D0245EB2403900106
:102650001124332339F030933E0287CF81E08093F9
:102660003D02F3CF81E080933E027FCF20910501B0
:102670008AE0289F900111242417350708F08BCF9A
:102680009F5F9093380202C09F3FD1F71D811123B5
:1026900059F00E943F119FEF11160CF491E0899FB1
:1026A000802D112480933F021E81112359F00E9436
:1026B0003F119FEF11160CF491E0899F802D11249A
:1026C0008093400230913F02332309F464CF20917C
:1026D0004002222309F45FCF45EB3403C0011124EB
:1026E000992359F090933F0245EB24039001112464
:1026F000332339F0309340024ECF81E080933F0284
:10270000F3CF81E08093400246CF83E290E00E94C5
:10271000F524833289F484E290E00E94F52483302A
:1027200059F485E290E00E94F52491E0893109F0A6
:1027300090E0892F8170089580E0FCCFCF93C82F5F
:102740006FEF811163E283E290E00E9403256FEF57
:10275000C11163E084E290E00E9403256FEFC11194
:1027600069E185E290E00E940325CF9108950895E4
:1027700086E290E00E94F524682F70E090E080E00F
:1027800008950895CF93C62F0E94C1136C2F86E23F
:1027900090E00E940325CF91089580E00E949E134F
:1027A00060E070E0CB010E94C2130E9484180E9476
:1027B000611981E00E949E1308950E94B7130E9440
:1027C000B8130E94C1130E948513811102C00E9498
:1027D000CD130895CF93FB01C281CC2309F19C0155
:1027E00022513F452031310520F582510E94711957
:1027F000C0E08C2FCF91089581E00E94690743E0EB
:1028000062E081E00E948602F3CF81E00E947507BA
:1028100043E062E081E00E948602EBCF82E0F6CFE7
:102820008031FFE59F0789F381319F45B9F3C1E00E
:10283000E0CF8031EFE59E07F9F281319F45C9F67F
:1028400082E0DBCF2FEFFC0120830895EF92FF920F
:102850000F931F93CF93DF93EC01062FE881E15094
:10286000E33108F05DC0F0E0EB5BFA4D0C94872497
:1028700019828AE08A83602FCE010E948B1DCDB71A
:10288000DEB7E6E00C94BC248981823069F08330A5
:1028900071F08130D9F40E94841C0E948D246A83D7
:1028A0007B838C839D83E7CF0E94B813F6CF7E0194
:1028B00082E0E80EF11C10E0812F0E94B50FF701B5
:1028C00081937F011F5F1530B9F7D5CF602FCE01FF
:1028D0000E942214D0CF89818230C1F76A817B8126
:1028E0008C819D810E948D240E94C213C4CF4B8194
:1028F0006A8189810E9446189827892798279D8395
:102900008C83B9CF2C813D813227232732274B81FD
:102910006A8189810E946818AECF0E948418ABCF6B
:102920008FEF8883A8CF0E9412198983A4CF0E94B9
:1029300014199827892798279A8389839CCF6B81BC
:1029400070E089819A81AE014C5F5F4F982789279B
:1029500098270E9417198FCF6B8170E089819A8127
:10296000AE014C5F5F4F9827892798270E943C193A
:1029700082CF0E9461197FCF0E943318D6CF6B811E
:1029800070E089819A81AE014C5F5F4F982789275B
:1029900098270E94BE186FCF6B8170E089819A8161
:1029A000AE014C5F5F4F9827892798270E94E11856
:1029B00062CFCF93DF93EC01FB018281882309F47E
:1029C00064C1C330FDE5DF07E0F5CA3F9CE5D907E8
:1029D00030F49E0122503C4524313105D8F50E9447
:1029E0003A0C9093770280937602C231ECE5DE07D1
:1029F00009F41FC108F06EC0C9308CE5D80709F48E
:102A0000F2C008F03FC0C530ECE5DE0709F4DBC0DA
:102A100058F5C3308CE5D80709F4CDC008F0CFC015
:102A2000809176028160C230DC4509F4AEC08091AD
:102A30007602909177020E94480C0E94E70680E09F
:102A400009C0C53AEDE5DE0751F238F4C1369DE51F
:102A5000D90729F2DF91CF9108959E012D5A3D4566
:102A600023303105B8F7BBCF809176028062C73042
:102A7000FCE5DF0709F489C008F4B1C08091760253
:102A8000806483C0CD309CE5D90709F4BAC070F4E6
:102A9000809176028E7FCB30FCE5DF0709F475C0AC
:102AA00008F4A7C0809176028D7F6FC0CF309CE57F
:102AB000D90709F4B6C008F4A8C0C031FCE5DF07A7
:102AC00009F4B3C0C131DC4509F0B1CF8091760281
:102AD0008F7B5BC0CF3F9CE5D90709F4B4C098F564
:102AE000CA3FFCE5DF0709F472C0B8F4C4319CE5C5
:102AF000D90709F4B6C008F4A2C0C531DC4509F015
:102B000096CF8091760282FB992790F921E0922757
:102B100090FB82F990FB83F938C0CC3F8CE5D80755
:102B200009F477C008F457C0CD3FECE5DE0709F49F
:102B300074C0809177028360CE3FDC4509F077CF87
:102B40008093770274CFC1368DE5D80709F496C01B
:102B500068F4C130EDE5DE0709F48CC008F477C0F5
:102B6000C230DD4509F063CF80E085C0CD3A9DE5F8
:102B7000D907E9F068F490917602892F8E7F90FF53
:102B80008160C53ADD4509F052CF809376024FCF80
:102B9000CE3A8DE5D80789F1CF3ADD4509F047CF28
:102BA00090917702892F877F93FF8860C9CF8091AA
:102BB00077028860C5CF809176028260E6CF8091EF
:102BC00076028460E2CF809176028860DECF8091C9
:102BD00077028160B5CF809177028260B1CF80911A
:102BE00076028061D2CF0E94E706809176028068EB
:102BF000CCCF809176028C60C8CF80917702877F9E
:102C00009FCF809176028B7FC0CF80917602877FA5
:102C1000BCCF809177028E7F93CF809177028D7F9A
:102C20008FCF809176028F7EB0CF809176028F7D9C
:102C3000ACCF0E94E706809176028F77A6CF809175
:102C40007602837FA2CF809177028C7F79CF8091AB
:102C50007702982F909591708E7F892B90FB81F948
:102C60006FCF0E94E70690917602892F97FB87F934
:102C700080588BCF81E00E94D40CD9CE90917602FF
:102C8000892F8F7E94FF806180CF81E0E3CEB0E01A
:102C9000A0E0EDE4F6E10C949F24E82FF0E0E45B83
:102CA000FE4FD490282F26952695269530E0F901E1
:102CB000E451FE4F0491877010E0082E02C0159574
:102CC00007950A94E2F701701127F901E452FE4FCB
:102CD000E490F12C082E02C0F594E7940A94E2F7F0
:102CE00091E0E922FF24F901E453FE4FC491D0E0C2
:102CF00002C0D595C7958A95E2F7C170DD27011509
:102D0000110519F081EE0E948303E114F10419F01A
:102D100086EE0E9483038D2D0E948A04E114F10443
:102D200019F086EE0E9419040115110519F081EEC3
:102D30000E941904CD2B19F08CE20E948A04CDB7B1
:102D4000DEB7E7E00C94BB24EF92FF920F931F9342
:102D5000CF93DF93EC01162F0AE08881882309F4D2
:102D600054C0813009F04EC08981813099F47E01D0
:102D700022E0E20EF11C8A810E948A04E70121967A
:102D8000812F815050F3EFE9FFE03197F1F700C058
:102D90000000F7CF823041F47E0182E0E80EF11CA2
:102DA0008A810E948303EACF833041F47E01E2E00E
:102DB000EE0EF11C8A810E941904E0CF843011F0DC
:102DC0002196DDCF2A81229690E080E0AE014F5F10
:102DD0005F4F2053330B2A30310548F0019778F2CA
:102DE000EFE9FFE03197F1F700C00000F7CF089F4F
:102DF000B001099F700D1124C901860F971F298109
:102E0000EA01E4CF0E944716BACFCDB7DEB7E6E0BD
:102E10000C94BC24EBEFE80FEF3308F062C0F0E055
:102E2000E85AFA4D0C9487240E94D10C81E0089551
:102E300080913002807F8093300281E08093440251
:102E400008950E94A502F2CF90913002892F8E7FC3
:102E500090FF81608093300280FDE8CF817F809376
:102E60003002E4CF90913002892F8D7F91FF8260F4
:102E70008093300281FFDACF809130028160EFCF02
:102E800090913002892F8B7F92FF84608093300273
:102E900082FDF2CFCBCF90913002892F877F93FFB5
:102EA00088608093300283FDE7CFC0CF0E94E706A1
:102EB00090917602892F97FB87F98058809376024C
:102EC000B5CF81E00E943A070E94E706AFCF895351
:102ED00091E001C0990F8A95EAF7892FF3CF8D51C0
:102EE000F7CF80E0089580E008950E947317089559
:102EF000CF93C82F809144028130B9F0882331F0FC
:102F00008230A1F11092440280E00DC00E94360B85
:102F10008232D1F78C2F0E94731781111BC08C2F26
:102F20000E940A178170CF9108950E94360B823259
:102F300089F38C2F0E94751781110AC0C43199F052
:102F400060F4CB3029F0C03169F782E0809344020D
:102F500081E0E8CF81E090E0E5CFC93221F0C833CD
:102F6000B9F380E0DFCF10924402FBCFC93209F4FD
:102F700040C0F0F4C431E9F1A8F481E0C73099F61B
:102F80008093090184E1809308018AE0809307011E
:102F90008EE18093060188E08093030188E28093AC
:102FA000020104C082EE8C0F8A3070F181E0BBCF49
:102FB000C03509F450C0B8F48AE0CF34B9F7E091D5
:102FC0004102F0914202309789F32081082E000CD3
:102FD000990B820F911D8F3F910509F00CF43FC0B2
:102FE0008FEF8083E3CFC135C1F181E0C23539F382
:102FF0009ACF809143028823C9F210924302109223
:10300000420210924102D2CFCD51C0934302C3304D
:10301000C9F048F4C13099F088E091E0C23051F035
:1030200010924302C3CFC53099F078F082E091E06E
:10303000C630B1F79093420280934102B7CF89E046
:1030400091E0F8CF87E091E0F5CF86E091E0F2CF14
:1030500083E091E0EFCF86EFB2CF8FEFB0CF97FF55
:10306000C0CF1082A3CF84E0089598E0699FB0019B
:10307000112450E0440F551F640F751F98E2899F7B
:10308000600D711D1124CB01879608950F931F9336
:10309000CF93DF938430C8F46530B8F44430A8F49B
:1030A0000E9435188C010E94F524C82FD0E0DC2F37
:1030B000CC27C80101960E94F5249E01282BC90146
:1030C000DF91CF911F910F91089590E080E0F8CFAC
:1030D0000F931F93CF93DF93122F032F843078F435
:1030E000653068F4443058F40E943518EC01602FC4
:1030F0000E940325612FCE0101960E940325DF91D6
:10310000CF911F910F910895B0E0A0E0EAE8F8E1B7
:103110000C949C248CEAC82E80E0D82ED0E0C0E02D
:10312000760110E01CC00E94180221E030E08C17EC
:103130001D0621F01CF0F50125913491402F612FDF
:103140008C2F0E94681882E0A80EB11C0F5F04301B
:1031500051F71F5F88E0E80EF11C153019F0570198
:1031600000E0E1CF219688E2C80ED11CC430D10521
:10317000B9F6CDB7DEB7EAE00C94B824EF92FF922F
:103180000F931F93CF93DF93EC018A017C01E60E2E
:10319000F71ECE018796CE15DF0529F4CDB7DEB731
:1031A000E6E00C94BC24C03AD10540F40E94F5241A
:1031B000F80180830F5F1F4F2196EBCFF80110823B
:1031C000F9CFB0E0A0E0E7EEF8E10C949E247C019A
:1031D0006A018C01060F171FEC01CE018796C017FC
:1031E000D10729F4CDB7DEB7E8E00C94BA24C03A91
:1031F000D10540F4FE01EE19FF09EC0DFD1D6081C3
:103200000E9403252196E9CF462F843040F4753083
:1032100030F4643020F4672F0E944618089590E03F
:1032200080E0089580E1089589E393E00895EF92A6
:10323000FF920F931F93CF93DF93EC018A017C01E0
:10324000E60EF71ECE0189539F4FCE15DF0529F4F8
:10325000CDB7DEB7E6E00C94BC24C93323E0D20737
:1032600040F40E94F524F80180830F5F1F4F2196E0
:10327000E9CFF8011082F9CFB0E0A0E0E2E4F9E193
:103280000C949E247C016A018C01060F171FEC012F
:10329000CE0189539F4FC017D10729F4CDB7DEB7B0
:1032A000E8E00C94BA24C93323E0D20740F4FE01CD
:1032B000EE19FF09EC0DFD1D60810E94032521968A
:1032C000E7CFCF93DF93C7ECD0E060E0CE010E9460
:1032D00003252196C11584E0D807B9F7DF91CF9176
:1032E0000895A4E0B0E0E7E7F9E10C949F24F82EFC
:1032F0008FE08F1548F18FEF93E00E94F524811144
:1033000023C007EC10E0F11023C019821A821B823F
:103310001C82DD24D39478018FEFE81AF80AC801E3
:103320000E94F52489831A82882371F09FEF980FF9
:103330009330D8F48A83D9820E5F1F4FC7010E9451
:10334000F5248B83811112C02496E7E00C94BB24F2
:10335000011584E01807C1F3C8010E94F52481110A
:1033600001C0FA940F5F1F4FCECF870160E0CE01FE
:1033700001960E94A416CFCFCF93DF93EB01863145
:103380009C4511F50E94360B9A81992399F08A7A0F
:1033900091E009F490E090934502811109C089E21F
:1033A0000E940E0B0E94770B80E0DF91CF91089571
:1033B00085E3F6CF80914502811104C089E20E9425
:1033C000160BF0CF85E3FBCF81E0EFCF0F931F9378
:1033D000CF93DF93C42FD22FFC0182818823C9F0C1
:1033E000409348020E94781C9093470280934602C3
:1033F00080E28C0F883040F4C77081E001C0880FF4
:10340000CA95EAF70E949304DF91CF911F910F9123
:10341000089510914802141332C080914602909191
:1034200047020E94901C883C910548F5C0E2CD0FF0
:103430001D17B9F080E2810F883040F4177081E0E9
:1034400001C0880F1A95EAF70E949A04C83048F420
:1034500081E09D2F977001C0880F9A95EAF70E942E
:103460009304802F0E948A04C83070F6D77081E0E0
:1034700001C0880FDA95EAF70E949A04C5CF80E26E
:103480008C0F883008F6C77081E001C0880FCA959C
:10349000EAF7F2CF0F939C01CB01233F4CE53407B1
:1034A00059F1A8F4283DFCE53F0701F1293D4CE521
:1034B0003407D1F1273D3C4591F406E221EE41EE7F
:1034C00067ED7CE50E94E61980E00F910895253FA5
:1034D000FCE53F07E9F0B0F0263F3C45F9F0FC0180
:1034E0008281882339F110924802EFCF07E225EE5E
:1034F00045EE68ED7CE5E6CF06E221EE40EE63EFB7
:103500007CE5E0CF07E225EE44EE64EF7CE5DACF20
:1035100006E221EE42EE65EF7CE5D4CF07E225EE30
:1035200046EE66EF7CE5CECF08E221E045EE69EDA0
:103530007CE5C8CF81E0C9CF90939301809392013D
:10354000089590934E0280934D020895E0914D02AC
:10355000F0914E02309729F00190F081E02D09950D
:10356000089580E00895E0914D02F0914E02309769
:1035700099F020911601222359F02091760227FF1D
:1035800007C0DC012C9111962C93119726E02C9307
:103590000280F381E02D09950895E0914D02F091AC
:1035A0004E02309739F022E0DC012C930480F58143
:1035B000E02D0995089520914B0230914C02281777
:1035C000390771F090934C0280934B02E0914D02C9
:1035D000F0914E02309721F00680F781E02D099599
:1035E00008952091490230914A022817390771F055
:1035F00090934A0280934902E0914D02F0914E026D
:10360000309721F00084F185E02D09950895FC01A3
:10361000329680911601882321F0809176029EE1F6
:1036200087FF96E080E0915008F4089521912223CD
:10363000D1F38F5FF8CF662301F120911601222389
:10364000F1F02091760227FF1AC0462F4695469545
:1036500046954E3190F4677021E030E002C0220FB1
:10366000331F6A95E2F7840F911DFC01828190E07F
:103670002823392381E0232B69F480E00895FC019D
:10368000329608962191261721F0E817F907D1F70D
:10369000F4CF81E008959C01FC0132969FEF80E019
:1036A0004191461751F09F3F19F4411101C0982FE5
:1036B0008F5F8630A9F79F3F09F40895290F311DC8
:1036C00097FD3A95F90162830895FC0132960896B8
:1036D0002191261303C0DF0111971C92E817F90707
:1036E000B9F70895E62FE695E695E695EE3168F48C
:1036F000E80FF92FF11D677021E030E001C0220FC3
:103700006A95EAF78281822B82830895E62FE695F7
:10371000E695E695EE3170F4E80FF92FF11D67702C
:1037200021E030E001C0220F6A95EAF720958281FE
:1037300028232283089520911601222339F0209115
:10374000760227FF03C00E94721B08950E944B1B44
:10375000089520911601222339F02091760227FF47
:1037600003C00E94861B08950E94651B0895FC01FA
:10377000329680911601882351F08091760287FF5E
:1037800006C08EE1DF011D928A95E9F7089586E073
:10379000F9CF46E050E00E94DF2421E0892B09F4B4
:1037A00020E0822F089508950E94D31B089581116F
:1037B00006C081E080934F020E94D41B089582E0EE
:1037C000F9CF83E080934F020E94D41B08950E949A
:1037D000D71B089581E080934F020E94D41B089567
:1037E0000E94EA1B0895089508950E94F41B08950D
:1037F000089508950E94F31B0895CF930E94F81B2B
:103800000E946D100E94F91BC0E08C2F0E94B50F22
:10381000811105C0CF5FC530C1F7CF91089581E018
:10382000FCCF85B7806885BF85B7806885BF089560
:103830001F921FB61F9211248F939F93AF93BF9334
:1038400080915002811113C0809182029091830275
:10385000A0918402B09185024196A11DB11D809373
:10386000820290938302A0938402B0938502BF9159
:10387000AF919F918F911F901FBE1F9018958091BF
:103880008A02843031F10E9409031092500288E1CB
:1038900090E020E40FB6F894A895809360000FBEE6
:1038A0002093600083B7817F846083BF83B781608A
:1038B00083BF7894889583B78E7F83BF0FB6F894C3
:1038C000A8958091600088618093600010926000EC
:1038D0000FBE08950E94E7060E940E03089582E03D
:1038E00084BD93E095BD9AEF97BD80936E000895D7
:1038F0002FB7F8948091820290918302A091840264
:10390000B09185022FBF08952FB7F894609182027D
:103910007091830280918402909185022FBF089557
:103920009C014FB7F8948091820290918302A091FC
:103930008402B09185024FBF821B930B0895789447
:103940001F921FB61F9211248F939F93AF93BF9323
:103950008091820290918302A0918402B0918502AD
:103960000196A11DB11D8093820290938302A093C2
:103970008402B0938502BF91AF919F918F911F9068
:103980001FBE1F90189581E08093E00080E2809335
:10399000D8001092C9008FE19EE40197F1F700C0B2
:1039A000000087E090EBDC018093930290939402F7
:1039B000A0939502B093960288E19CE00FB6F8942C
:1039C000A895809360000FBE90936000FFCF88E1C0
:1039D0009CE00FB6F894A895809360000FBE90937A
:1039E0006000FFCF80917402089508959C0184E0E7
:1039F0008093E9009FEF8091E800915085FD06C01B
:103A000085ED8A95F1F700009111F5CF8091E800DE
:103A100085FF0CC050E040E066E070E0C9010E9404
:103A20009D1F8091E8008E778093E8000895CF93E2
:103A3000DF93EC01809116018823B1F18091760229
:103A400087FF32C060E284E08093E9008FEF9091BD
:103A5000E800815095FD06C095ED9A95F1F70000BC
:103A60008111F5CF8091E80085FF1BC08091160180
:103A700070E050E040E0811104C050E040E068E0B8
:103A800070E0CE010E949D1F8091E8008E778093A8
:103A9000E80080E2FE01A4E5B2E001900D928A9573
:103AA000E1F7DF91CF91089568E081E0CDCF809379
:103AB0005102709353026093520280918A028430C3
:103AC000F9F48093E9008FEF9091E800815095FD23
:103AD00006C095ED9A95F1F700008111F5CF809120
:103AE000E80085FF0DC050E040E063E070E081E554
:103AF00092E00E949D1F8091E8008E778093E800FD
:103B00000895BC0184E00E94571D0895BC0183E024
:103B10000E94571D0895CF93FC01603221F58091DA
:103B20008A02843001F5C091E900CF702091EC0049
:103B3000922F917020FD90E8C92B82E08093E900DC
:103B40008091E80080FF0CC050E040E060E270E04F
:103B5000CF010E949D1F8091E8008E778093E8003E
:103B6000CF70C093E900CF910895809189028111AF
:103B700009C00E947C210E94D9218091E2008460CA
:103B80008093E20008951092890208950E94EA1B32
:103B900008956091860281E0611101C080E00E9479
:103BA000E11B089590918A0281E0943009F080E051
:103BB000609186020E94E71B089542E061EC81E07B
:103BC0000E94F82042E261EC84E00E94F82042E288
:103BD00061EC82E00E94F82042E260EC83E00E9407
:103BE000F82090918A0281E0943009F080E06091A1
:103BF00086020E94D71B089580918C02833009F4BD
:103C000063C030F48130E1F1823009F4A0C008953E
:103C10008A3009F48CC08B3009F471C0893009F006
:103C200052C080918B02813209F04DC080918F0289
:103C300090919002009719F0029709F044C080918A
:103C4000E800877F8093E8008091E80082FF37C01A
:103C50009091F3008091F200029731F48091F1008D
:103C6000813011F0863021F48091F100809374024C
:103C70008091E8008B778093E8000E942C2123C07C
:103C800080918B02813AF9F48091E800877F8093DC
:103C9000E80080918F0290919002892B61F460E29C
:103CA00084E592E070E00E943B208091E8008B77F1
:103CB0008093E800089560E090E080E0F3CF809189
:103CC0008A028111C1CF089580918B02813AD9F780
:103CD00080918F0290919002892BA9F78091E80042
:103CE000877F8093E8008091E80080FFFCCF80917F
:103CF00016018093F1008091E8008E77BCCF80910F
:103D00008B02813201F780918F0290919002892B72
:103D1000D1F68091E800877F8093E8000E942C21F3
:103D200080918D02809316010E94E706089580918C
:103D30008B02813241F68091E800877F8093E80012
:103D40000E942C2180918E028093750208958091AB
:103D50008B02813A09F0B7CF8091E800877F80938A
:103D6000E8008091E80080FFFCCF80917502C1CF10
:103D700084B7877F84BF0FB6F894A89580916000C0
:103D8000886180936000109260000FBE80E890E030
:103D90000FB6F89480936100909361000FBE0E946B
:103DA000F01B08950E947C210E94D921E2EEF0E0F0
:103DB00080818460808378940E94582408958AE0EA
:103DC00091E00E94A11A089580918A02853031F411
:103DD00080918A02853019F00E946A1C08950E9421
:103DE0003F1C80918802882399F30E94FD1B882341
:103DF00079F30E94871F0E94E706EACFA0E2B0E0B5
:103E0000E4E0FFE10C94A42480918A02843009F557
:103E100083E08093E9008091E80082FF1AC08091DE
:103E2000E80090E085FF09C050E040E060E270E00B
:103E3000CE0101960E94EC1F91E08091E8008B7703
:103E40008093E800992329F060E2CE0101960E9458
:103E50002614A096E2E00C94C0240E94301F08951E
:103E6000292F33272330310521F168F42130310522
:103E700009F443C02230310509F444C090E080E0E9
